 AdvBacklight

 Timestamp is 4da2a52e (Mon Apr 11 18:52:30 2011)

 Preferred load address is 10000000

 Start         Length     Name                   Class
 0001:00000000 0000017aH .rdata                  CODE
 0001:0000017c 00000029H .rdata$debug            CODE
 0001:000001a8 00000b58H .text                   CODE
 0001:00000d00 00000028H .idata$2                CODE
 0001:00000d28 00000014H .idata$3                CODE
 0001:00000d3c 00000048H .idata$4                CODE
 0001:00000d84 0000001aH .idata$6                CODE
 0001:00000da0 00000056H .edata                  CODE
 0002:00000000 00000048H .idata$5                DATA
 0002:00000048 00000038H .bss                    DATA
 0003:00000000 00000048H .pdata                  DATA
 0004:00000000 000000a0H .rsrc$01                DATA
 0004:000000a0 00000228H .rsrc$02                DATA

  Address         Publics by Value              Rva+Base       Lib:Object

 0000:00000000       ___safe_se_handler_count   00000000     <absolute>
 0000:00000000       ___safe_se_handler_table   00000000     <absolute>
 0001:00000098       ??_C@_1DC@DOOLNADC@?$AAC?$AAh?$AAa?$AAn?$AAg?$AAe?$AA?5?$AAe?$AAv?$AAe?$AAn?$AAt?$AA?5?$AAt?$AAr?$AAi?$AAg?$AAg?$AAe?$AAr?$AAe?$AAd?$AA?$AN?$AA?6?$AA?$AA@ 10001098     advbacklight_common_topaz_v1:advbacklight.obj
 0001:000000cc       ??_C@_1DE@PFEDGFDL@?$AAB?$AAa?$AAc?$AAk?$AAL?$AAi?$AAg?$AAh?$AAt?$AAL?$AAe?$AAv?$AAe?$AAl?$AAC?$AAh?$AAa?$AAn?$AAg?$AAe?$AAE?$AAv?$AAe?$AAn?$AAt?$AA?$AA@ 100010cc     advbacklight_common_topaz_v1:advbacklight.obj
 0001:00000100       ??_C@_1EC@GCKNHFJA@?$AAR?$AAe?$AAa?$AAd?$AA?5?$AAT?$AAr?$AAa?$AAc?$AAk?$AAB?$AAa?$AAr?$AA?3?$AA?5?$AAb?$AAa?$AAt?$AAt?$AA?$DN?$AA?$CF?$AAd?$AA?5?$AAE?$AAx?$AAt?$AA?$DN?$AA?$CF?$AAd?$AA?5?$AA?$AN?$AA?6@ 10001100     advbacklight_common_topaz_v1:advbacklight.obj
 0001:00000144       ??_C@_1DG@KBMJFALH@?$AAR?$AAe?$AAs?$AAt?$AAo?$AAr?$AAe?$AA?3?$AA?5?$AAb?$AAa?$AAt?$AAt?$AA?$DN?$AA?$CF?$AAd?$AA?5?$AAE?$AAx?$AAt?$AA?$DN?$AA?$CF?$AAd?$AA?5?$AA?$AN?$AA?6?$AA?$AA@ 10001144     advbacklight_common_topaz_v1:advbacklight.obj
 0001:000001a8       BacklightAdvApplet         100011a8 f   advbacklight_common_topaz_v1:advbacklight.obj
 0001:000003a8       DllEntry                   100013a8 f   advbacklight_common_topaz_v1:advbacklight.obj
 0001:00000410       ?AdvancedDlgProc@@YAHPAUHWND__@@IIJ@Z 10001410 f   advbacklight_common_topaz_v1:advbacklight.obj
 0001:0000070c       ?GetFromRegistry@@YAXPAK0PBG11@Z 1000170c f   advbacklight_common_topaz_v1:advbacklight.obj
 0001:000007a8       ?SetToRegistry@@YAXPAK0PBG11@Z 100017a8 f   advbacklight_common_topaz_v1:advbacklight.obj
 0001:0000083c       ?InitSliders@@YAXPAUHWND__@@KK@Z 1000183c f   advbacklight_common_topaz_v1:advbacklight.obj
 0001:00000960       ?UpdateBklSettings@@YAXPAUHWND__@@@Z 10001960 f   advbacklight_common_topaz_v1:advbacklight.obj
 0001:00000b04       ?RestoreBklSettings@@YAXKK@Z 10001b04 f   advbacklight_common_topaz_v1:advbacklight.obj
 0001:00000bcc       SetEvent                   10001bcc f i advbacklight_common_topaz_v1:advbacklight.obj
 0001:00000c00       LocalFree                  10001c00 f   coredll:COREDLL.dll
 0001:00000c10       LocalAlloc                 10001c10 f   coredll:COREDLL.dll
 0001:00000c20       GetWindowLongW             10001c20 f   coredll:COREDLL.dll
 0001:00000c30       SendMessageW               10001c30 f   coredll:COREDLL.dll
 0001:00000c40       GetDlgItem                 10001c40 f   coredll:COREDLL.dll
 0001:00000c50       SetWindowLongW             10001c50 f   coredll:COREDLL.dll
 0001:00000c60       RegCloseKey                10001c60 f   coredll:COREDLL.dll
 0001:00000c70       RegQueryValueExW           10001c70 f   coredll:COREDLL.dll
 0001:00000c80       RegOpenKeyExW              10001c80 f   coredll:COREDLL.dll
 0001:00000c90       RegSetValueExW             10001c90 f   coredll:COREDLL.dll
 0001:00000ca0       CloseHandle                10001ca0 f   coredll:COREDLL.dll
 0001:00000cb0       CreateEventW               10001cb0 f   coredll:COREDLL.dll
 0001:00000cc0       NKDbgPrintfW               10001cc0 f   coredll:COREDLL.dll
 0001:00000cd0       EventModify                10001cd0 f   coredll:COREDLL.dll
 0001:00000ce0       PropertySheetW             10001ce0 f   commctrl:commctrl.dll
 0001:00000cf0       __rt_udiv                  10001cf0 f   corelib1:COREDLL.dll
 0001:00000d00       __IMPORT_DESCRIPTOR_COREDLL 10001d00     coredll:COREDLL.dll
 0001:00000d14       __IMPORT_DESCRIPTOR_commctrl 10001d14     commctrl:commctrl.dll
 0001:00000d28       __NULL_IMPORT_DESCRIPTOR   10001d28     coredll:COREDLL.dll
 0002:00000000       __imp_LocalFree            10002000     coredll:COREDLL.dll
 0002:00000004       __imp_LocalAlloc           10002004     coredll:COREDLL.dll
 0002:00000008       __imp_GetWindowLongW       10002008     coredll:COREDLL.dll
 0002:0000000c       __imp_SendMessageW         1000200c     coredll:COREDLL.dll
 0002:00000010       __imp_GetDlgItem           10002010     coredll:COREDLL.dll
 0002:00000014       __imp_SetWindowLongW       10002014     coredll:COREDLL.dll
 0002:00000018       __imp_RegCloseKey          10002018     coredll:COREDLL.dll
 0002:0000001c       __imp_RegQueryValueExW     1000201c     coredll:COREDLL.dll
 0002:00000020       __imp_RegOpenKeyExW        10002020     coredll:COREDLL.dll
 0002:00000024       __imp_RegSetValueExW       10002024     coredll:COREDLL.dll
 0002:00000028       __imp_CloseHandle          10002028     coredll:COREDLL.dll
 0002:0000002c       __imp_CreateEventW         1000202c     coredll:COREDLL.dll
 0002:00000030       __imp_NKDbgPrintfW         10002030     coredll:COREDLL.dll
 0002:00000034       __imp_EventModify          10002034     coredll:COREDLL.dll
 0002:00000038       __imp___rt_udiv            10002038     corelib1:COREDLL.dll
 0002:0000003c       \177COREDLL_NULL_THUNK_DATA 1000203c     coredll:COREDLL.dll
 0002:00000040       __imp_PropertySheetW       10002040     commctrl:commctrl.dll
 0002:00000044       \177commctrl_NULL_THUNK_DATA 10002044     commctrl:commctrl.dll
 0002:00000048       ?rgPropPages@@3PAU_PROPSHEETPAGEW@@A 10002048     advbacklight_common_topaz_v1:advbacklight.obj
 0002:0000004c       ?PropHdr@@3U_PROPSHEETHEADERW@@A 1000204c     advbacklight_common_topaz_v1:advbacklight.obj
 0002:00000074       ?g_hInst@@3PAUHINSTANCE__@@A 10002074     advbacklight_common_topaz_v1:advbacklight.obj

 entry point at        0001:000003a8

 Static symbols

